:100000000C9446000C9465000C9465000C946500FB
:100010000C9465000C9465000C9465000C946500CC
:100020000C9465000C946E000C9465000C946500B3
:100030000C9465000C9465000C9465000C946500AC
:100040000C9465000C9465000C9465000C9465009C
:100050000C9465000C9465000C9465000C9465008C
:100060000C9465000C9465000C9465000C9465007C
:100070000C9465000C9465000C9465000C9465006C
:100080000C9465000C9469030C94650011241FBE48
:10009000CFEFD0E1DEBFCDBF11E0A0E0B1E0EEEAEE
:1000A000FBE000E00BBF02C007900D92A430B10747
:1000B000D9F712E0A4E0B1E001C01D92A031B10770
:1000C000E1F70E94C4000C94D5050C9400008BE06D
:1000D00085BD89EF83BD80E887BF08951F920F9289
:1000E0000FB60F9211248F939F93AF93BF9380917C
:1000F000040190910501A0910601B09107010196BC
:10010000A11DB11D8093040190930501A0930601E8
:10011000B0930701BF91AF919F918F910F900FBE48
:100120000F901F901895EF92FF920F931F9383B338
:1001300098E0892785BB80910101909102018C593B
:100140009F4F9093020180930101885E934030F0AD
:1001500088EC90E0909302018093010100910101ED
:100160001091020186E9E82EF12C20E030E040E019
:1001700050E060E070E083E990E00E9422011F916E
:100180000F91FF90EF900895EF92FF920F931F93BE
:10019000F8940E9434030E94670087E080930F0266
:1001A00060E070E080E090E00E94460378948FEF7A
:1001B00084BB22E3E22EF12C00E61AEE21E030E0CF
:1001C00040E050E060E070E08AEF90E00E942201A1
:1001D00096E9E92EF12C08EC10E020E030E040E058
:1001E00050E060E070E083E990E00E9422010E940C
:1001F0001A02FDCF8091000185BB60E67AEE8AEF9E
:1002000090E00E94A8020895FC01838994890297D6
:10021000C1F48281803361F0813399F48FEF809350
:10022000000160E67AEE8AEF90E00E94A80208954D
:1002300083818093000160E070E08AEF90E00E948B
:10024000A8020895CF92DF92EF92FF920F931F932F
:10025000CF93DF93EC016B01A0E0B0E09A2FFD019A
:1002600084E0EE0FFF1F8A95E1F7EA0FFB1FE85FBE
:10027000FE4F8785882329F09F5F1196AC30B1052A
:1002800069F7692F70E0FB01A4E0EE0FFF1FAA954C
:10029000E1F7E60FF71FE85FFE4FD183C083D382FB
:1002A000C2825583448337832683E114F10411F419
:1002B000108A08C082E3E816F10411F481E001C05D
:1002C00082E0808BFB0134E0EE0FFF1F3A95E1F7EF
:1002D000E60FF71FE85FFE4FA089B0E0AC52BE4FBB
:1002E0008C91982F9E0D96878F5F8C931187008736
:1002F00081E08787F89420910401309105014091B5
:10030000060150910701C801A0E0B0E0820F931FE1
:10031000A41FB51FFB0124E0EE0FFF1F2A95E1F794
:10032000E60FF71FE85FFE4F82879387A487B587A4
:100330007894DF91CF911F910F91FF90EF90DF9014
:10034000CF900895CF92DF92EF92FF920F931F9379
:10035000CF93DF93DC01EB01690120E030E0622FF5
:10036000F90174E0EE0FFF1F7A95E1F7E20FF31F3A
:10037000E85FFE4F8785882331F06F5F2F5F3F4F27
:100380002C30310561F7262F30E0F90164E0EE0FE3
:10039000FF1F6A95E1F7E20FF31FE85FFE4FB1839D
:1003A000A083D383C28355834483D782C682E1145A
:1003B000F10411F4108A08C082E3E816F10411F484
:1003C00081E001C082E0808BB90194E0660F771F65
:1003D0009A95E1F7620F731F685F7E4FEB01E88922
:1003E000F0E0EC52FE4F8081982F9E0D9E878F5F2C
:1003F00080831987088781E08F87209104013091DD
:1004000005014091060150910701C801A0E0B0E04C
:10041000820F931FA41FB51FFB0182879387A487B8
:10042000B587DF91CF911F910F91FF90EF90DF90F3
:10043000CF900895EF92FF920F931F93CF93DF9386
:10044000F894E0900401F0900501009106011091EC
:10045000070178941092D7018091DA018F5F809321
:10046000DA018091DA01883C49F48091D9018695BE
:100470008093D8011092D9011092DA014FEF5FEF0B
:1004800020E030E0F901A4E0EE0FFF1FAA95E1F7AC
:10049000E20FF31FE85FFE4F8785882399F0809174
:1004A000D7018F5F8093D70182859385A485B58519
:1004B000E816F9060A071B0728F08685851710F449
:1004C0005685422F2F5F3F4F2C303105D9F64F3FD5
:1004D000B9F18091D9018F5F8093D901842F992739
:1004E00087FD9095EC01E4E0CC0FDD1FEA95E1F784
:1004F000C80FD91FC85FDE4FE881F9816C817D810B
:100500008A819B8109958E819F81892B49F41F8661
:10051000E889F0E0EC52FE4F80818150808310C06A
:100520002A853B854C855D8588859985A0E0B0E06E
:10053000820F931FA41FB51F8A879B87AC87BD8737
:1005400081E0DF91CF911F910F91FF90EF9008957F
:100550009C01DB0160E070E0FB0144E0EE0FFF1F57
:100560004A95E1F7E60FF71FE85FFE4F8081918122
:100570008217930719F58785882301F1F894209154
:100580000401309105014091060150910701CD0110
:10059000A0E0B0E0820F931FA41FB51FFB0124E071
:1005A000EE0FFF1F2A95E1F7E60FF71FE85FFE4FFA
:1005B00082879387A487B587789408956F5F7F4F6C
:1005C0006C30710549F60895AC0120E030E0F90186
:1005D000A4E0EE0FFF1FAA95E1F7E20FF31FE85F1B
:1005E000FE4F8081918184179507B9F48785882310
:1005F000A1F0209104013091050140910601509134
:100600000701CB01A0E0B0E0820F931FA41FB51F2C
:1006100082879387A487B58708952F5F3F4F2C303B
:100620003105A9F60895AC0120E030E0F901B4E00D
:10063000EE0FFF1FBA95E1F7E20FF31FE85FFE4FE1
:10064000808191818417950749F41786E089F0E04D
:10065000EC52FE4F80818150808308952F5F3F4F81
:100660002C30310519F7089580E090E0FC0124E07A
:10067000EE0FFF1F2A95E1F7E80FF91FE85FFE4F25
:10068000178601968C30910589F7089580910F02A5
:10069000880F81608093720080E480937000E1E7AE
:1006A000F0E080818C7F80832FEF2093730085ECB6
:1006B0008093740081E090E09093DE018093DD01EF
:1006C0001092DC01209309021092F3011092F201C2
:1006D00008951F920F920FB60F920BB60F9211242E
:1006E000EF92FF920F931F932F933F934F935F933C
:1006F0006F937F938F939F93AF93BF93EF93FF93EA
:100700008091DD019091DE01817C09F4CBC0809164
:10071000710090E0887F90708038910561F1813898
:100720009105ACF48836910509F48AC089369105A3
:100730002CF48036910509F0B3C09AC0803791053A
:1007400009F496C08837910509F0AAC079C08039AC
:10075000910589F0813991052CF48838910509F0CB
:100760009FC096C08839910509F492C0803A9105DE
:1007700009F096C093C08091DD019091DE01803434
:10078000910581F4809173008093E0018FEF809355
:10079000090280E890E09093DE018093DD011092E1
:1007A000DC017CC08091DD019091DE0180389105F3
:1007B00009F074C09091DC018091E0019817A0F4D9
:1007C0008091DC01E82FF0E090917300E152FE4F40
:1007D00092838F5F8093DC01909109028091730076
:1007E0008927809309025AC08091DC01803111F57C
:1007F000809173008093F101909109028091F10141
:10080000981719F081E090E002C082E090E09093A8
:10081000F3018093F201EE24FF2400E010E020E0D9
:1008200030E040E050E06FED71E084E091E00E9444
:10083000A2012EC08091DC018F5F8093DC012EC06D
:1008400080910D028F5F80930D0280910A028A30A1
:1008500078F422E3E22EF12C02E310E020E030E015
:1008600040E050E060E070E08EE395E00E94A2017D
:10087000809173008093DF011092F3011092F201D6
:100880001092DC0185EC8093740080E490E07DC0E0
:1008900081E090E09093DE018093DD0185ECD5C08E
:1008A00085E4D3C08091710090E0887F90708032A1
:1008B000910509F49CC08132910554F48031910571
:1008C00099F088319105D1F0089709F0B7C00CC0B4
:1008D0008033910509F45EC08833910509F460C046
:1008E000889709F0ABC011C08091F4018093730028
:1008F00085E88093740088E090E047C01092DB01A7
:100900008091F501809373003BC08091DB018131C0
:10091000D9F485E98093740080E290E09093DE0141
:100920008093DD0110920A0280910B0290910C02DB
:10093000019690930C0280930B0260E070E086E4D5
:1009400093E00E94E40283C09091DB018091F50165
:10095000981750F080910602809373008091DB011C
:100960008F5F8093DB010CC09091DB01E92FF0E0F9
:10097000EC50FE4F8281809373009F5F9093DB0168
:1009800085E88093740080E190E09093DE0180938D
:10099000DD015DC080910D028F5F80930D022CC040
:1009A00080910D028F5F80930D0260E070E086E41D
:1009B00093E00E94E40280910A028A3080F492E37C
:1009C000E92EF12C02E310E020E030E040E050E0BE
:1009D00060E070E08EE395E00E94A20106C088E22C
:1009E00090E09093DE018093DD0185E82EC0809138
:1009F0000E028F5F80930E0260E070E086E493E069
:100A00000E94E40280910A028A3080F482E3E82E98
:100A1000F12C02E310E020E030E040E050E060E044
:100A200070E08EE395E00E94A20106C088E290E0AB
:100A30009093DE018093DD0185E907C084E090E0BA
:100A40009093DE018093DD0185E080937400FF9137
:100A5000EF91BF91AF919F918F917F916F915F9136
:100A60004F913F912F911F910F91FF90EF900F9019
:100A70000BBE0F900FBE0F901F901895EF92FF9234
:100A80000F931F938091DD019091DE01019771F02A
:100A900042E3E42EF12C05E010E020E030E040E0FD
:100AA00050E060E070E08EE395E01DC01092DB0145
:100AB00085EA8093740082E090E09093DE01809359
:100AC000DD0180910A028F5F80930A0232E3E32EF8
:100AD000F12C00E117E220E030E040E050E060E07F
:100AE00070E086E493E00E9422011F910F91FF9035
:100AF000EF900895EF92FF920F931F93582F8091DC
:100B00000A02882309F448C080910A028A3009F455
:100B100043C081E03CC08FEF80930602DB0120E000
:100B200030E00DC08C91F901EC50FE4F8283809132
:100B300006029D918927809306022F5F3F4F24175D
:100B400088F381E080930A02852F90E0880F991F37
:100B50008093F4014093F5011092DB0185EA8093C4
:100B6000740082E090E09093DE018093DD0152E317
:100B7000E52EF12C05E010E020E030E040E050E010
:100B800060E070E086E493E00E94220180E01F9123
:100B90000F91FF90EF9008958091DD019091DE011B
:0E0BA000019709F4B8CF82E0F2CFF894FFCFAE
:040BAE00FFC800007C
:00000001FF
